:100000004DEF0FF068961200046ED8CF05F0E0CFE8
:1000100006F00001E9CF0CF0EACF07F0E1CF08F0DD
:10002000E2CF09F0D9CF0AF0DACF0BF0F3CF12F01C
:10003000F4CF13F0FACF14F000C00EF001C00FF0AF
:1000400002C010F003C011F0A0AA2AEF00F0A1BA7C
:10005000FAEF07F00EC000F00FC001F010C002F080
:1000600011C003F00CC0E9FF07C0EAFF078E08C00B
:10007000E1FF09C0E2FF0AC0D9FF0BC0DAFF12C0DE
:10008000F3FF13C0F4FF14C0FAFF045006C0E0FFF2
:1000900005C0D8FF1000F76AA60FF66E000EF72213
:1000A0000900F5501200000302FFFFFFFFFFFFFFF2
:1000B000FFFFFFFFFFFFF76AC60FF66E000EF72285
:1000C0000900F550120000FF02FFFFFFFFFFFFFFD6
:1000D000FFFFFFFFFFFFF76AE60FF66E000EF72245
:1000E0000900F550120040000B0040000000000025
:1000F0000000000000000000000000000000000000
:1001000000000000000007AE03D0F2CF0DF0F29E19
:10011000F76A280FF66E010EF7220900F55007AEB8
:1001200002D00DBEF28E1200400000004000000020
:1001300000000000000000000000000000000000BF
:100140000000000000000000F76A580FF66E010E74
:10015000F7220900F5501200090243000201008055
:10016000320904000001020201000524001001040C
:10017000240202052406000105240100010705816F
:10018000030B00FA09040100020A0000000705023F
:10019000024000010705820240000100F76AAC0F2F
:1001A000F66E010EF7220900F55012000200F76A00
:1001B000BE0FF66E010EF7220900F550120012175D
:1001C0001B20FFFFFFFFF76AD60FF66E010EF72226
:1001D0000900F550120012011001020000406104F4
:1001E0003300000101020001F76AF80FF66E010EFC
:1001F000F7220900F5501200040309040803430024
:1002000044004300180355005300420020007400CE
:100210006F00200055004100520054006D92699417
:1002200068A402D06894FCD706EF08F0400E0401E1
:10023000016F040E036F180E026F880E006F046BBF
:10024000040E076F580E066F0001120070A002D056
:10025000EDDF7090689A0DEF08F06A6A689212EF0D
:1002600008F0C291C1BFC281C19FC151100803E211
:10027000000E016E20D0C2A110D0036AC151F2CF8E
:10028000C3F0F29E08DFC3BFF28EFF0802E1000E4A
:1002900001D0010E016E0FD00ED0036AC151F2CF12
:1002A000C3F0F29E08DFC3BFF28EFF0802E1000E2A
:1002B00001D0010E016E1200C651C803F3CF01F048
:1002C000F4CF00F0C903F3500026C751C803F35020
:1002D0000020026E1200036AC051700FE96E0F0E0B
:1002E0000320EA6EEF6AC0C0C1F0BBDF015222E01A
:1002F000C76BC0C0C6F0C96B080EC86FDDDF01C098
:10030000E9FF040E0224EA6EEF6AC76BC0C0C6F0B4
:10031000C96B080EC86FD0DF02C0C2F001C0C1F0C7
:10032000040EC127000EC223C1C0E9FF040EC2257E
:10033000EA6EEF6A1200010EBF6FBF510F0805E3AE
:10034000BFC0C0F0C8DFBF2BF8D71200B96BB86BC5
:10035000250EB76F800EB66FEA6A2E0EE96EE26A5E
:10036000B60EE16E020E016EE6CFEEFF012EFCD757
:10037000306A316AB66BEA6A320EE96EE26AB60E2C
:10038000E16EE6CFEEFFB66BEA6A330EE96EE26A23
:10039000B60EE16EE6CFEEFF080EB66FEA6A340ED7
:1003A000E96EE26AB60EE16EE6CFEEFF806B7F91FA
:1003B000366A356A7E6B2190816B12002B6A2A6A3D
:1003C000B56BB55101080AE3036AB5512C0FE96E0C
:1003D000000E0320EA6EEF6AB52BF3D7B7DF1B6A76
:1003E000010E1C6E1A6A12006A6A686A9F0E6B6EB2
:1003F0003D0E696E6E6A9FDFE1DF160E706E68A6B5
:1004000002D000DEFCD76D9811DF030E256E17EFCA
:1004100008F0698468986D821CEF08F0689C21EFF1
:1004200008F0BAC026F0120026681200B86B2A50F5
:100430002B103CE0B8513F0839E31D5005E0020A9B
:100440000EE0010A17E020D029C003F02850F2CFB7
:10045000BAF0F29E79DEBABFF28EB96F15D029C01C
:1004600003F02850F2CFBAF0F29EBEDEBABFF28E91
:10047000B96F0AD029C003F02850F2CFBAF0F29E2B
:10048000A2DEBABFF28EB96F282AD8B4292A2A5020
:10049000D8B42B062A06B851B82B580FE96E040EB3
:1004A000EA6ED8B0EA2AB9C0EFFFC1D72A502B10A4
:1004B00004E1B851400801E01A6AB8C0BAF0B1DFEF
:1004C0001200296A286A1D6A04011B51010A0001F1
:1004D00007E0030A0BE0010A0DE0220A27E049D0F9
:1004E0002B6A120E2A6E030E1D6E45D02B6A430E28
:1004F0002A6E41D0020E1D6E036A04011A511E0FAE
:10050000E96E000E0320EA6E296AEFCF28F029C0B9
:1005100003F02850F2CFB7F0F29E000165DEB7BFBE
:10052000F28E036A2A6E03C02BF025D0036A040101
:100530001A51F2CFB7F0F29E000139DEB7BFF28E4A
:10054000036A286E03C029F0283C02D029520FE02C
:1005500029C003F02850F2CFB7F0F29EF5DDB7BF07
:10056000F28E036A2A6E03C02BF005D002D05CDF46
:1005700011D05ADF0FD004011F5308E12B5203E1C1
:100580002A501E5D03E22B6A1EC42AF0010E1A6E69
:1005900000014CDF10EF04F0B75304E1040E256EA8
:1005A000CADEE9D0050E256E040EBA6F980EB96F3B
:1005B000010EB86FB8510F08D8A0DDD0B8C0C0F098
:1005C0008ADEBB6B036AB851F2CFBFF0F29E73DDD7
:1005D000BFBFF28EFF0865E0040EBB6FD890B83540
:1005E000036AF2CFBFF0F29E8EDD0900F5CF03F073
:1005F000BFBFF28EBC6F03C0BDF0C76BB8C0C6F002
:10060000C96B080EC86F58DE01C0BFF0010E01248F
:10061000016E000E0220036E01C0E9FF040E0324E8
:10062000EA6EBCC0EFFFC76BB8C0C6F0C96B080E5E
:10063000C86F42DE01C0BFF0020E0124016E000E41
:100640000220036E01C0E9FF040E0324EA6EBAC063
:10065000ECFFED52B9C0EFFFD890B835036AF2CF86
:10066000BFF0F29E50DD0900F5CF03F0BFBFF28E60
:10067000B9270350BA23880EBE6FBDA101D0BE8139
:10068000BDA301D0BE83C76BB8C0C6F0C96B080E4E
:10069000C86F12DE01C0E9FF040E0224EA6EBEC07C
:1006A000EFFF036AB851F2CFBFF0F29EF4DCBFBF98
:1006B000F28EFF0845E0BB83C76BB8C0C6F0C96BBC
:1006C000080EC86FF9DD02C0C0F001C0BFF0040E13
:1006D000BF27000EC023020EBF25016E000EC021F1
:1006E000036E01C0E9FF040E0324EA6EBAC0ECFFFA
:1006F000ED52B9C0EFFFD890B835036AF2CFBFF022
:10070000F29EE9DC0900F5CF03F0BFBFF28EB927F6
:100710000350BA23C76BB8C0C6F0C96B080EC86FC8
:10072000CBDD02C0C0F001C0BFF0040EBF27000E39
:10073000C023BFC0E9FF040EC025EA6E400EEF6E75
:10074000BB51060802E10E0EBB6F036AB851F2CF2F
:10075000BFF0F29EA0DCBFBFF28E010801E0BB89B2
:10076000036AB851700FE96E0F0E0320EA6EBBC02A
:10077000EFFFB82B1FD70AEF04F004011951000A4C
:1007800000010DE0010A14E0020A1FE0060A29E058
:10079000030A2EE00E0A2EE0010A32E040D01CC00F
:1007A00058F40401596B020E0001BA6F3ADE38D0DA
:1007B00004011A2D07D0010E1C160001BA6B31DEA0
:1007C00003D00401000130DE2BD004011A2D06D025
:1007D0001C820001BA6B25DE03D00401000124DE77
:1007E0001FD0020E1A6E1AC427F0BA6B1ADE18D088
:1007F00068D616D01BC058F4010EBA6F12DE10D0A6
:1008000004011A51010809E31AC41BF01AC4B7F015
:100810000001C2D6BA6B05DE0401000101D004DE7E
:1008200085EF05F01BC0B7F004011951000A000163
:1008300005E00A0A0BE0010A2BE03CD00401586BEA
:10084000596B020E0001BA6FECDD35D0B7531EE0D4
:10085000010EB75D036AF2CFB8F0F29E9FDCB8BF1D
:10086000F28E016E04011C5DD8A002D000010ED0F2
:10087000036A1C512C0FE96E000E0320EA6EEFCFC5
:1008800058F4010E0001BA6FCCDD01D0CDDD13D0DC
:10089000B7530EE0036A04011C512C0FE96E000EE1
:1008A0000320EA6E1AC4EFFF0001BA6BBADD01D073
:1008B000BBDD01D0B9DD85EF05F0B891B7BFB881D8
:1008C000B79FB8A117D0C76BB7C0C6F0C96B080EE9
:1008D000C86FF2DC02C0BAF001C0B9F0040EB9274B
:1008E000000EBA23B9C0E9FF040EBA25EA6E880EDD
:1008F000EF6E0DD0C76BB7C0C6F0C96B080EC86FDE
:10090000DBDC01C0E9FF040E0224EA6EEF6AFDEFB2
:1009100004F0B891B7BFB881B79FB8A117D0C76B23
:10092000B7C0C6F0C96B080EC86FC6DC02C0BAF00B
:1009300001C0B9F0040EB927000EBA23B9C0E9FF0F
:10094000040EBA25EA6E840EEF6E0ED0C76BB7C0E8
:10095000C6F0C96B080EC86FAFDC01C0E9FF040E1A
:100960000224EA6E840EEF6E03EF05F0B891B7BF74
:10097000B881B79FB8A117D0C76BB7C0C6F0C96B15
:10098000080EC86F99DC02C0BBF001C0BAF0040EBB
:10099000BA27000EBB23BAC0E9FF040EBB25EA6EDE
:1009A000EFCFB9F00ED0C76BB7C0C6F0C96B080E59
:1009B000C86F82DC01C0E9FF040E0224EA6EEFCFAB
:1009C000B9F0B9AF02D0B9B502D0000E01D0010E16
:1009D000016E0DEF05F01CC4C1F043DC015228E0AC
:1009E00004011951010A000105E0020A09E0030AA5
:1009F0000DE01DD01CC4B7F060D7BA6B12DD18D063
:100A00001CC4B7F086D7BA6B0CDD12D00401586B4A
:100A1000596B1CC4B7F00001A9D7015204E0010EC4
:100A20000401586F0001020EBA6FFBDC01D0FCDC40
:100A300085EF05F0FE0E266E120004011C2D01D07C
:100A400002D01C5348E11951000A00010BE0010AD1
:100A50000DE0210A1CE0010A1FE0030A2EE0010A52
:100A600031E037D0010E816FE5DF34D0040EEA6E3D
:100A7000580EE96EE26A370EE16E080E016EE6CF9F
:100A8000EEFF012EFCD71EC4BAF0CBDC23D0020E41
:100A9000816F7F81CFDF1ED0040EEA6E580EE96EA3
:100AA000E26A2E0EE16E070E016EE6CFEEFF012E1A
:100AB000FCD7070EBA6FB5DC0DD01AC480F0BA6B44
:100AC000B0DC08D01AC436F01BC435F0BA6BA9DC10
:100AD00001D0AADC0401000185EF05F01A6A0401C7
:100AE00018517F0B000A000107E0010A07E0030A22
:100AF00007E0230A07E008D040D607D093D605D0F8
:100B00006AD703D09AD701D08FDCB0EF07F0C76B5C
:100B1000B8C0C6F0C96B080EC86F5CEC01F001C02C
:100B2000E9FF040E0224EA6EEFCFBAF0B9510208D1
:100B300006E1BAAD02D0B96B02D0010EB96FB9515E
:100B400003081AE1840EBA6FC76BB8C0C6F0C96B50
:100B5000080EC86F5CEC01F002C0BEF001C0BDF031
:100B6000040EBD27000EBE23BDC0E9FF040EBE2546
:100B7000EA6E840EEF6E07D0B92D03D0C80EBA6F9F
:100B800002D0880EBA6FD890B835036AF2CFBDF0A4
:100B9000F29E83EC00F00900F5CF03F0BDBFF28EAA
:100BA000BB6F03C0BCF0C76BB8C0C6F0C96B080E02
:100BB000C86F5CEC01F001C0BDF0010E0124016EB4
:100BC000000E0220036E01C0E9FF040E0324EA6E4A
:100BD000BBC0EFFFBCA101D0BA81BCA301D0BA83D6
:100BE000C76BB8C0C6F0C96B080EC86F5CEC01F0EB
:100BF00001C0E9FF040E0224EA6EBAC0EFFF120042
:100C0000036AC551700FE96E0F0E0320EA6EEF52B2
:100C100019E0C76BC5C0C6F0C96B080EC86F5CECA5
:100C200001F002C0C7F001C0C6F0040EC627000ED6
:100C3000C723C6C0E9FF040EC725EA6EEFCFC8F090
:100C4000C8AF02D0000E01D0010E016E1200C0C06C
:100C5000C5F0D6DF0152D8B47DD0C76BC0C0C6F096
:100C6000C96B080EC86F5CEC01F002C0C6F001C091
:100C7000C5F0040EC527000EC623010EC525016E62
:100C8000000EC621036E01C0E9FF040E0324EA6EC4
:100C9000C1C0EFFFC35102081EE1C76BC0C0C6F060
:100CA000C96B080EC86F5CEC01F002C0C6F001C051
:100CB000C5F0040EC527000EC623C5C0E9FF040E0B
:100CC000C625EA6EEFCFC4F0C4AD02D0C36B02D02C
:100CD000010EC36F18D0C351040815E1C76BC0C023
:100CE000C6F0C96B080EC86F5CEC01F001C0E9FFEB
:100CF000040E0224EA6EEFCFC4F0C4AD03D0010E9F
:100D0000C36F01D0C36BC32D03D0C80EC46F02D014
:100D1000880EC46FC2A101D0C481C2A301D0C48314
:100D2000C76BC0C0C6F0C96B080EC86F5CEC01F0A1
:100D300002C0C6F001C0C5F0040EC527000EC623D0
:100D4000C5C0E9FF040EC625EA6EC4C0EFFF010E60
:100D5000016E02D0000E016E12008151010A03E003
:100D6000030A13E024D0EA6A370EE96E040EE26E3D
:100D7000180EE16E080E016EE6CFEEFF012EFCD7D5
:100D8000BA6B11EC02F0816B13D0EA6A2E0EE96E99
:100D9000040EE26E180EE16E070E016EE6CFEEFF56
:100DA000012EFCD7816BBA6B11EC02F001D0816B84
:100DB0000DEF07F0C76BB8C0C6F0C96B080EC86F5F
:100DC0005CEC01F002C0BAF001C0B9F0010E0124E0
:100DD000016E000E0220036E01C0E9FF040E032421
:100DE000EA6E036AEFCF01F003C002F003EF07F0F1
:100DF0002190020EB86FB96F8ADE12002180236A3B
:100E0000020EB86FD7D701C022F0225201E1F0DF05
:100E100012EF07F0B75302E1A0D704D0B751020890
:100E200001E1ECD71200B8C06EFFB85303E0040E26
:100E3000256E02D0020E256E23EF07F01B6A1A6A98
:100E400027C0B8F0F0D78FEF07F0B8C0C5F0D8DEF4
:100E5000015243E0C76BB8C0C6F0C96B080EC86F3B
:100E60005CEC01F002C0C1F001C0C0F0040EC0276C
:100E7000000EC123020EC025016E000EC121036EBB
:100E800001C0E9FF040E0324EA6EECCFBFF0ED527F
:100E9000EFCFBEF0BFC0EAFFBEC0E9FFBAC0E2FFBD
:100EA000B9C0E1FFBCC002F0BBC001F0015202E0DA
:100EB000022A02D0025206E0E6CFEEFF012EFCD756
:100EC000022EFAD7B8C0C0F0BCC0C2F0BBC0C1F09F
:100ED000BDC0C3F0BCDE015002D0000E016E120096
:100EE0007E530EE0020EB86FBA6B3F0EB96FBC6B4B
:100EF0007EC0BBF0020EBD6FA8DF015201E07E6B29
:100F00001200EEDF94EF07F0B7530AE11A2C03D07A
:100F100016EC02F004D01A500208D8B48FD704D0CF
:100F2000B751020801E1EDD712002430B56FB53397
:100F3000B5331F0EB517245241E1040100513C0B9B
:100F40000001B66F430E040100170001B6513408CA
:100F50001EE104010451800B01E0046B0001BED5C9
:100F60006D98263C05D0B86B030EB96FD0DD0ED05E
:100F7000B86B020EB96FCBDD2650FE0807E0C06BE0
:100F8000C26B26C0C1F0040EC36F61DE16D0B6512D
:100F9000040813E1B76B3EDFB86B020EB96FB7DD23
:100FA0002650FE080AE0263C01D007D0C06BC26B79
:100FB00026C0C1F0010EC36F4ADE1AD024500408C7
:100FC0000EE12668B76BA0DF263C01D007D0C06BCE
:100FD000C26B26C0C1F0020EC36F39DE09D024B443
:100FE00004D0B5C0B7F016DF03D0B5C0B7F08CDFC2
:100FF0002BEF08F0A19A2552D8B433D06852D8B458
:1010000030D068A403D069B40EEF01F06DB229D0DE
:1010100068AA03D069BA26EF01F068A203D069B2CA
:101020002DEF01F068A003D069B0F4EF01F068A8DB
:1010300003D069B809EF02F068AC03D069BC0EEFC9
:1010400002F0B46B68A608D069A606D06CCF24F075
:1010500002EC00F06AD701D004D0B451B42B0308DD
:10106000F1E22AEF00F00A54544D5342202D204E55
:101070006F7765456E65726769652E6F72670A00E6
:101080000A54544D5342202D204E6F7765456E65AE
:10109000726769652E6F72670A000A6461790000E1
:1010A0000A6D6F6E746800000A79656172000A68E3
:1010B0006F7572000A6D696E00000A73656B00003F
:1010C0006D6A696A080E6F6E94503009946E256AD5
:1010D000166AF2BE168EF29EDEEC01F016BEF28E9D
:1010E00073EF08F0EDD770EF0FF09C6B9C51070881
:1010F0001BE393968A96070E006E002EFED700D053
:10110000D8909B3302E28A9601D08A869396EF0E9E
:10111000006E002EFED700D09386070E006E002EC4
:10112000FED700D09C2BE2D71200010E9D5F0CE38E
:10113000EA6A9D0EE96EEF5007E0020E006E002E87
:10114000FED700D0EF2EF9D7120093968A96020EA2
:101150009B6FFA0E9D6FE9DF9B2FFBD79386020EE4
:101160009B6FFA0E9D6FE1DF9B2FFBD793861200DA
:10117000EA6A9B0EE96EEF500EE00F0E016E006AF8
:10118000002EFED7012EFBD78F0E006E002EFED74D
:101190000000EF2EF2D71200166AF2BE168EF29EF3
:1011A000DEEC01F016BEF28E6D6A140E6F6E696A87
:1011B0006D86010E256EE0EF08F06DB601D0ECD71C
:1011C000252C0BD06DBA09D0686A696AA08AC00E56
:1011D000F212110E696E020E256E94EF0FF01B5085
:1011E000016E44EF09F00900F5520DE0F6CF95F0DD
:1011F000F7CF96F0F5509EA8FED7AD6E95C0F6FFDE
:1012000096C0F7FFF0D767EF09F0A291A0BAA281CC
:10121000A09A7E513E0802E23E0E7E6F7E517E2BEA
:10122000036A3F0FE96E000E0320EA6EA1C0EFFFD4
:10123000A09AA2B1A08A20EF09F0A0C0A1F0E5D742
:10124000166AF2BE168EF29E4BDE16BEF28E30EF9E
:1012500009F07E513E0801E2FCD79FC0A0F0EDD717
:1012600012000900F5520CE0F6CF95F0F7CF96F09A
:10127000F5CF9FF0EEDF95C0F6FF96C0F7FFF1D7F0
:101280001200010E926FABD701C093F0946B7FB147
:10129000942B935303E096948D9402D096948D846E
:1012A000945303E096948D9402D096948D8480A1FB
:1012B00003D094908B9002D094908B8094530CE048
:1012C00090530AE1660EF66E100EF76E8CD7800E04
:1012D000F66E100EF76EC5DF92C08EF093C08FF0E1
:1012E00094C090F096EF0FF021B001D0FDD72350BD
:1012F000232AA30FE96E040EEA6ED8B0EA2AEFCFD4
:1013000093F02250235C07E3166AF2BE168EF29E1B
:101310006FDD16BEF28E93C001F012008251660896
:1013200005E195908C806E0E826F04D095908C9024
:10133000660E826FC1EF0FF096948D94020E926F3D
:10134000960E9B6F15DF922FFBD796948D84020E1D
:10135000926F960E9B6F0CDF922FFBD796948D9415
:10136000020E926F960E9B6F03DF922FFBD796941F
:101370008D8412008351660805E195928C826E0E71
:10138000836F04D095928C92660E836FC6EF0FF038
:1013900093988A88040E926FFA0E9B6FE9DE922F63
:1013A000FBD793988A983AEF10F095968C8695948F
:1013B0008C84640E9B6FDCDE95968C9695948C9451
:1013C0003AEF10F095968C8695988C88640E9B6FFA
:1013D000CFDE95968C9695988C983AEF10F0959C68
:1013E0008C8C959E8C8E640E9B6FC2DE959C8C9C23
:1013F000959E8C9E3AEF10F0959C8C8C959A8C8AD9
:10140000640E9B6FB5DE959C8C9C959A8C9A3AEFF6
:1014100010F09951016A985D03E298C000F00CD079
:10142000006A080E9A6F983700369951005CD8B060
:10143000006E01369A2FF7D7120093C098F00A0E6B
:10144000996FE7DF0150100DF3CF94F093C098F03F
:101450000A0E996FDEDF00509425016E1200080E0F
:10146000016E110E006E002EFED78A929392110E1D
:10147000006E002EFED798378A90D8B09380D8A0FF
:101480009390938281A2FED7012EEBD7110E006EAE
:10149000002EFED78A92939200009380110E006E68
:1014A000002EFED7110E006E002EFED7938281A271
:1014B000FED7016A110E006E002EFED781B00180AA
:1014C0008A9293928A90939012009380110E006EEC
:1014D000002EFED79382110E006E002EFED78A904A
:1014E0009390110E006E002EFED78A929392D00E2A
:1014F000986FB5DF94C098F0B2DF95C098F0AFDF79
:1015000093900000938281A2FED7110E006E002EF0
:10151000FED700D000009380110E006E002EFED783
:101520009380110E006E002EFED79382110E006E76
:10153000002EFED78A909390110E006E002EFED7DB
:101540008A929392D00E986F8ADF0150969101B0E3
:101550009681976B96B103D0975104081DE3938051
:10156000110E006E002EFED79382110E006E002E1B
:10157000FED781A2FED78A909390110E006E002EA6
:10158000FED78A929392D00E986F69DF01509691A0
:1015900001B09681972BDED712009A0EF66E100ED0
:1015A000F76E5FDEA1DE01C092F092C093F045DFDE
:1015B00001C093F0040E946F01C095F086DFA00E79
:1015C000F66E100EF76E4DDE8FDE01C092F092C007
:1015D00093F033DF01C093F0050E946F01C095F0D6
:1015E00074DFA80EF66E100EF76E3BDE7DDE01C0D6
:1015F00092F092C093F021DF01C093F0060E946F39
:1016000001C095F062DFAE0EF66E100EF76E29DEA9
:101610006BDE01C092F092C093F00FDF01C093F037
:10162000020E946F01C095F050DFB40EF66E100EEE
:10163000F76E17DE59DE01C092F092C093F0FDDE26
:1016400001C093F0010E946F01C095F03EDFBA0E19
:10165000F66E100EF76E05DE47DE01C092F092C006
:1016600093F0EBDE01C093F0946B01C095F02DDF99
:10167000DAEF0FF0080E956F00C096F09380110E10
:10168000006E002EFED7938281A2FED781B0D88053
:1016900081A0D8900136110E006E002EFED79392D5
:1016A0008A92952FEBD79380110E006E002EFED7F5
:1016B0008A909651D8A493900000938281A2FED77D
:1016C000110E006E002EFED78A929392110E006EBC
:1016D000002EFED78A909390A1EF0BF09380110E0D
:1016E000006E002EFED79382110E006E002EFED7E4
:1016F00081A2FED78A909390110E006E002EFED725
:101700008A929392D00E986FAADE92C098F0A7DECC
:101710009380110E006E002EFED79382110E006E84
:10172000002EFED781A2FED78A909390110E006EF4
:10173000002EFED78A929392D10E986F90DE006AA7
:1017400099D701C093F093900000938281A2FED7B5
:10175000110E006E002EFED700D000009380110EF7
:10176000006E002EFED793C001F012009339006E78
:101770000F0E001600500A0DF3CF94F093510F0B8B
:101780009425016E1200926BA9DF01C092F001C096
:1017900093F0ECDF01C088F0010E926F9FDF01C073
:1017A00092F001C093F0E2DF01C089F0020E926F67
:1017B00095DF01C092F001C093F0D8DF01C08AF03C
:1017C000040E926F8BDF01C092F001C093F0CEDF68
:1017D00001C08BF0050E926F81DF01C092F001C055
:1017E00093F0C4DF01C08CF0060E926F77DF01C06A
:1017F00092F001C093F0BADF01C08DF0DFEF0FF07F
:10180000200E93A9300E946F92C000F092AF08D0D2
:10181000001E002A00C092F02D0E946F938F9381CA
:10182000015092C098F0640E996FF3DD00C092F001
:10183000300E0124956F92C098F00A0E996FE9DD81
:10184000300E0024976F300E0124966F94C000F084
:10185000300E955D04E0938393BF938512D094C0BE
:1018600095F0200E946F300E965D04E0938193BF47
:10187000938307D0D8A4938104E195C096F0200EFD
:10188000956F93B505D093B306D093B107D009D027
:1018900094C09FF0DEDC95C09FF0DBDC96C09FF02B
:1018A000D8DC97C09FF0D5DC12009B6B9B510708DA
:1018B00019E393968A96070E006E002EFED700D08D
:1018C00093861F0E006E002EFED700D0938681B641
:1018D00002D0D89001D0D8809C33780E9D6F25DC43
:1018E0009B2BE4D79CC001F012008E0E006E9CC0B2
:1018F00001F09BC002F0036A9CAF05D0011E021EDE
:10190000022A01E1012A015209E102C001F0026A42
:10191000080E005E015202E1006A0AD0D89001BEB2
:1019200004D0023601360006F9D79CBF01D0019ED3
:101930007FEF0DF09F51D8B4A5D0AB6FA351D8B4B1
:10194000A1D0AB5F05E37F0EAB27D8B09BD006D00C
:10195000810EAB5FD8A096D0D8B494D0ABC000F0C5
:10196000016A026A036AAA6BA0C0A9F0A98FA1C08C
:10197000A8F0A2C0A7F0190EAB6FA651A75F0DE2A9
:10198000010EA85F0AE2A95F08E2AA5F06E2AA2B9D
:10199000A92BA82BA651A72728D0A551A85F12E2F2
:1019A000010EA95F0FE2AA5F0DE2AA2BA92BA55198
:1019B000A827A651A72719E3A82B17E1A92B15E102
:1019C000AA2B13D0A4518009A95F0EE2010EAA5FD1
:1019D0000BE2AA2BA4518009A927A551A827E9E366
:1019E000A92BE7E1AA2BE5D70380AB2F01D00BD0C1
:1019F000D890A737A837A937AA37D8900336023628
:101A00000136AC37BAD7ACA106D0D8900132023239
:101A10000332AC3302D0000635E0ACBF1ED0D89004
:101A2000A737A837A937AA37A651A75F07E2010E43
:101A3000A85F04E2A95F02E2AA5F1AE3A551A85FCA
:101A400005E2010EA95F02E2AA5F12E3A451800938
:101A5000A95F03E2010EAA5F0BE3032A09E1022A50
:101A600007E1012A05E1002A0DE0013202320332CA
:101A7000A0C0ABF0A451AB1BABAF02D0018E06D01F
:101A8000019E04D0006A016A026A036A95EF0DF0B4
:101A9000926BA5EC08F0CC0E9B6F75EC08F0440E31
:101AA0009B6F75EC08F0C80E9B6FB8EC08F0925372
:101AB00004E1FBDE01C092F0FAD7A5EC08F0CC0EF1
:101AC0009B6F75EC08F0BE0E9B6F75EC08F0EDDEB9
:101AD00001C093F0EADE01C094F0E7DE01C017F028
:101AE000E4DE01C018F0E1DE01C019F094C096F008
:101AF00093C095F096C09CF095C09BF0F6D603C0BD
:101B00009EF002C09DF001C09CF000C09BF003C09D
:101B1000A2F002C0A1F001C0A0F000C09FF0A66B2F
:101B2000A56BA46B830EA36F05D703C09AF002C008
:101B300099F001C098F000C097F0C80E9B6FB8EC08
:101B400008F097C000F098C001F099C002F09AC068
:101B500003F017EF10F09F51D8B471D0006EA3516D
:101B6000D8B46DD0002604E3810E002668E204D0CC
:101B70007F0E005E64E363E0A0C0A7F0A451A71B42
:101B8000A08FA48FA251A603F4CFA9F0A151A50361
:101B9000F4CF03F0F3CFA8F0A603F350A927F45035
:101BA000A823000E0322A251A503F350A927F45045
:101BB000A823000E026A03220222A051A603F350BA
:101BC000A827F4500322000E0222A051A503F350CF
:101BD0000326F4500222000E016A0122A251A4033E
:101BE000F350A827F4500322000E02220122A15133
:101BF000A403F3500326F4500222000E0122A05148
:101C0000A403F3500226F4500122002A01BE05D09D
:101C1000A8370336023601360006000EA8AF0AD0F8
:101C2000032A02220122015005E1025003E1035080
:101C300001E1002AA7BF018EA7AF019E04D0006A70
:101C4000016A026A036AA0EF0EF09F51B6089F6F07
:101C5000036AA0C0A3F0A08FD890A033A133A23311
:101C600003320232013200329F2FF6D7A3AF0BD0DE
:101C7000001E011E021E031E002AD8B4012AD8B479
:101C8000022AD8B4032AB3EF0EF0D8B203D0EA6A1E
:101C9000A70EE96E006A016A026A036AA76BA86B65
:101CA000A96BAA6BA651A511A411A3112CE0200EBB
:101CB000AB6FD8909F37A037A137A237A737A83787
:101CC000A937AA37A651AA5D08E1A551A95D05E18A
:101CD000A451A85D02E1A351A75D0FE3A351A75F43
:101CE000A451D8A0A43DA85FA551D8A0A53DA95F47
:101CF000A651D8A0A63DAA5FD8800036013602368C
:101D00000336AB2FD6D7A7C0EFFFA8C0ECFFA9C002
:101D1000ECFFAAC0ECFF1200E950976F9651996F43
:101D200019E095C0A2F094C0A1F093C0A0F092C0B9
:101D30009FF0A66BA56B200EA46F820EA36F0BD72E
:101D400003C095F002C094F001C093F000C092F07F
:101D5000992FE7D795C0A2F094C0A1F093C0A0F04E
:101D600092C09FF072D703C095F002C094F001C0FA
:101D700093F000C092F095AF0DD09707978B921F0C
:101D8000931F941F951F922BD8B4932BD8B4942BE8
:101D9000D8B4952B3B0E9E6F9A0E9D6FCA0E9C6F0A
:101DA0009B6B0A0E996F9651D8B4972BD882EA6A2A
:101DB000920EE96E95C0A2F094C0A1F093C0A0F07D
:101DC00092C09FF09EC0A6F09DC0A5F09CC0A4F05C
:101DD0009BC0A3F05ADF015000520FE19629995D94
:101DE0000CE097510CE00F0B995D01E03BE297BFCF
:101DF00039D097BD04D0200E30D0200E971797AB66
:101E00000DD0979B9651D8A497070050976F2D0E31
:101E10009F6F29EC09F09751006E976B9651995D71
:101E20000BE10050976F2E0E9F6F29EC09F0975130
:101E3000006E200E9717000E300E97AB0ED0979BBA
:101E40009651D8A497070050976F2D0E9F6F29ECDD
:101E500009F09751006E976B300E002600C09FF07E
:101E600029EC09F0D8929EC0A2F09DC0A1F09CC0C0
:101E7000A0F09BC09FF0A66BA56BA46B0A0EA36F8E
:101E800004DF03C09EF002C09DF001C09CF000C0C2
:101E90009BF0992F8BD72CEF10F0F86AD09E078E0D
:101EA000B886E10EAF6E040EB06EA60EAC6E900E4C
:101EB000AB6E660E826F836FC150C00B0F09C16E8F
:101EC000070EB46E1E6A040E1F6E0C0E206E8E6B13
:101ED0008F6B906B96948D8494908B8072EF08F04A
:101EE000CC0E9B6F75EC08F04E0E9B6F75EC08F0F6
:101EF0007D0E9B6F75EC08F0C90E9B6F75EC08F0BA
:101F00007F0E9B6F75EC08F0A5EC08F0CC0E9B6F74
:101F100075EC08F0480E9B6F75EC08F00F0E9B6F88
:101F2000B8EC08F0DDEF08F041EF09F09EAA08D008
:101F30009EAAFED7AECF91F091C09FF029EC09F098
:101F400021A098D074EC09F001C091F091516D0A74
:101F500016E0030A19E01D0A1CE0060A1DE0110A3A
:101F60001EE0080A1FE01E0A20E01D0A21E0160AF2
:101F700024E00D0A5BE0040AD8B471D07BD08EEF68
:101F800009F09CEC09F076D0BAEF09F09CEC09F06E
:101F900071D0C8EF09F06ED0D5EF09F06BD0E2EF49
:101FA00009F068D0EFEF09F065D0FCEF09F062D0DE
:101FB000CDEF0AF09CEC09F05DD0C3EF0BF08BC0C5
:101FC00092F0180E936F1CDC2D0E9F6F29EC09F018
:101FD0008CC092F0180E936F13DC2D0E9F6F29ECBE
:101FE00009F08DC092F0180E936F0ADC200E9F6FDF
:101FF00029EC09F08AC092F0180E936F01DC3A0EBA
:102000009F6F29EC09F089C092F0180E936F00ECD5
:102010000CF03A0E9F6F29EC09F088C092F0180E70
:10202000936F00EC0CF09CEC09F024D031D503C088
:1020300087F002C086F001C085F000C084F0020E77
:10204000E96E87C095F086C094F085C093F084C097
:1020500092F0010E966F60D69CEC09F00BD06F0EDB
:102060009F6F29EC09F06B0E9F6F29EC09F09CEC37
:0820700009F000D057D703006E
:020000040030CA
:0E00000024CE3E1E0087A1000FC00FE00F406F
:00000001FF
